:020000040000FA
:04000000CC303A289E
:08000800A000030EA100831209
:100010008B1C32288B1031181428B11C3228643004
:10002000010203183128182800001628172818285C
:1000300019281A281B281C281D281E281F283110A3
:10004000B114A810031005190314AA0DA90DA80DC9
:10005000B00B322831152A08AF002908AE00280855
:10006000AD00B11081010B11210E8300A00E200EF6
:02007000090085
:0C007400203084008001840A6030040207
:10008000031C3C281230B000AD2183160C308505CE
:1000900087018312850187010730990000309A009B
:1000A000103083168E008312603083168F00831207
:1000B0000030831691008312C830831681008312AA
:1000C00031309000003083168C00831210308B008A
:1000D000831600309B001C141A088312BC00831680
:1000E00010309B001C141A088312BD003E228101AF
:1000F0008E018F010B118B100B108C018B178E2032
:100100003119A420B30B8C28031085190314B90DE1
:10011000F03039020319262195227F286400311816
:1001200008000B1D08000B11B11031141230B00083
:10013000051D9F2832148316011383120800321004
:10014000831601178312080031110130B7008B1399
:100150002030370783169B001C141A088312A40052
:10016000A500C030A5061030370783169B001C146D
:100170001A088312A3000030370783169B001C1453
:100180001A088312A2008B17321CCC2822090339CB
:10019000A200A309A409A50922082D02031D2029F4
:1001A00023082E02031D202924082F02031D2029C5
:1001B00001303702031DE1283D18E1283D143E14AB
:1001C000BA2102303702031DEA28BD18EA28BD14FF
:1001D0003E14C62103303702031DF3283D19F328CE
:1001E0003D153E14D22104303702031DFC28BD19F1
:1001F000FC28BD153E14DE2105303702031D0529FC
:100200003D1A05293D163E14EA2106303702031D2A
:100210000E29BD1A0E29BD163E14F52107303702EE
:10022000031D17293D1B17293D173E1400220830D6
:100230003702031D2029BD1B2029BD173E140B22A8
:10024000B70A0930370203180800A7280130B600A2
:10025000B300B400B500B70085018701B1138E204B
:10026000B30B5E29031085190314B90DF030390260
:1002700003198529B40B5E290130370203191622B0
:100280000230370203191B220330370203192022E0
:1002900004303702031925220530370203192A22B8
:1002A0000630370203192F22073037020319342290
:1002B00008303702031939229630B400311D2F2936
:1002C0003111321C68292D090339AD00AE09AF097F
:1002D0002F1CB1132F1C2F29B11B2F292E182F29AA
:1002E000B1178B1320303707BB002F08BA009821B5
:1002F00010303707BB002E08BA00982100303707AE
:10030000BB002D08BA0098218B1785018701B70A19
:10031000B60109303702031C2F293E2208003E1C7B
:1003200008003E101030BB003D08BA0098210800BC
:100330008B133A0883161C159A0083123B08831608
:100340009B0055309D00AA309D009C1464009C18B1
:10035000A6291C1183128B170800FF30C800CA158C
:10036000CB15CC15CD15CE15CF15D015D115D21571
:10037000D3150800F130BD05FF30DE051130C4058E
:10038000C0000030C200C6005F100800F230BD059A
:10039000FF30DE050230C405C0000030C200C600D8
:1003A0005F100800F430BD05FF30DE050630C405DF
:1003B000C0000030C200C6005F100800F830BD0564
:1003C000FF30DE051830C405C0000030C200C60092
:1003D0005F1008001F30BD05C030DE058830C50540
:1003E000C1000030C300C70008002F30BD05C03079
:1003F000DE051030C505C1000030C300C70008008D
:100400004F30BD05C030DE053030C505C1000030BD
:10041000C300C70008008F30BD05C030DE05C03006
:10042000C505C1000030C300C700080010308506B4
:100430000230870608002030850600308706080055
:10044000213085060030870608000230850602301C
:1004500087060800003085060C308706080000304B
:1004600085060130870608000030850621308706A2
:100470000800003085061830870608003D18BA21AC
:10048000BD18C6213D19D221BD19DE213D1AEA2130
:10049000BD1AF5213D1B0022BD1B0B220800B60131
:1004A000B301B4013C1C572ABC01BC14592ABC013D
:1004B0003C143C08B60064005D2A5E2A5F2A602A6C
:1004C000612AFF30B41B8500B41F8501B30B5B2A82
:1004D000B40B5B2A0310B60CB608031D5B2A003070
:1004E000BB003C08BA009821080005125C180516EC
:1004F000DC1C8512DC1885165C1D05105C190514C2
:10050000DC1D8510DC1985145C1E87105C1A8714AD
:10051000DC1E0711DC1A07155C1F07105C1B071493
:10052000DC1F8712DC1B871608008F0803190800E0
:100530008F0178308E00C80FBF2CC80A441CC52A12
:10054000461CB62ACA1CA72ACA014A15D32A4A1D24
:10055000AC2ACA01CA15D32ACA1DB12ACA014A1631
:10056000D32A4A1ED32ACA01CA14D32A4A1DBB2A37
:10057000CA014A16D32ACA1DC02ACA014A16D32A5A
:100580004A1ED32ACA01CA14D32ACA1CCA2ACA01BB
:100590004A15D32A4A1DCF2ACA01CA15D32A4A1E90
:1005A000D32ACA014A15C41CFA2AC61CEB2ACB1C42
:1005B000DC2ACB014B15082B4B1DE12ACB01CB15B7
:1005C000082BCB1DE62ACB014B16082B4B1E082B04
:1005D000CB01CB14082B4B1DF02ACB014B16082B5B
:1005E000CB1DF52ACB014B16082B4B1E082BCB013C
:1005F000CB14082BCB1CFF2ACB014B15082B4B1D12
:10060000042BCB01CB15082B4B1E082BCB014B1514
:10061000441D2F2B461D202BCC1C112BCC014C151F
:100620003D2B4C1D162BCC01CC153D2BCC1D1B2B73
:10063000CC014C163D2B4C1E3D2BCC01CC143D2B3C
:100640004C1D252BCC014C163D2BCC1D2A2BCC014F
:100650004C163D2B4C1E3D2BCC01CC143D2BCC1C01
:10066000342BCC014C153D2B4C1D392BCC01CC151A
:100670003D2B4C1E3D2BCC014C15C41D652BC61DBE
:10068000562BCD1C472BCD014D155F13732B4D1DE4
:100690004C2BCD01CD15732BCD1D512BCD014D16FE
:1006A000732B4D1E732BCD01CD14732B4D1D5B2B66
:1006B000CD014D16732BCD1D602BCD014D16732B27
:1006C0004D1E732BCD01CD14732BCD1C6A2BCD0188
:1006D0004D15732B4D1D6F2BCD01CD15732B4D1E5D
:1006E000732BCD014D155F1B9C2B441E9C2B461E6E
:1006F0008D2BCE1C7E2BCE014E15AA2B4E1D832B8F
:10070000CE01CE15AA2BCE1D882BCE014E16AA2BBC
:100710004E1EAA2BCE01CE14AA2B4E1D922BCE011B
:100720004E16AA2BCE1D972BCE014E16AA2B4E1E6F
:10073000AA2BCE01CE14AA2BCE1CA12BCE014E1576
:10074000AA2B4E1DA62BCE01CE15AA2B4E1EAA2BD0
:10075000CE014E15C51DD12BC71DC22BCF1CB32BEF
:10076000CF014F15DF2B4F1DB82BCF01CF15DF2B3E
:10077000CF1DBD2BCF014F16DF2B4F1EDF2BCF011F
:10078000CF14DF2B4F1DC72BCF014F16DF2BCF1DF3
:10079000CC2BCF014F16DF2B4F1EDF2BCF01CF14F9
:1007A000DF2BCF1CD62BCF014F15DF2B4F1DDB2BA3
:1007B000CF01CF15DF2B4F1EDF2BCF014F15451E6D
:1007C000062C471EF72BD01CE82BD0015015142CFB
:1007D000501DED2BD001D015142CD01DF22BD001C3
:1007E0005016142C501E142CD001D014142C501D53
:1007F000FC2BD0015016142CD01D012CD00150160A
:10080000142C501E142CD001D014142CD01C0B2CE2
:10081000D0015015142C501D102CD001D015142CC3
:10082000501E142CD0015015C51E3B2CC71E2C2C5D
:10083000D11C1D2CD1015115492C511D222CD10147
:10084000D115492CD11D272CD1015116492C511EEF
:10085000492CD101D114492C511D312CD1015116F3
:10086000492CD11D362CD1015116492C511E492C31
:10087000D101D114492CD11C402CD1015115492C46
:10088000511D452CD101D115492C511E492CD101A6
:100890005115451F712C471F622CD21C532CD201BD
:1008A0005215DF137F2C521D582CD201D2157F2CEC
:1008B000D21D5D2CD20152167F2C521E7F2CD201EC
:1008C000D2147F2C521D672CD20152167F2CD21DC0
:1008D0006C2CD20152167F2C521E7F2CD201D214C6
:1008E0007F2CD21C762CD20152157F2C521D7B2CD2
:1008F000D201D2157F2C521E7F2CD2015215DF1B44
:10090000A82CC51FA82CC71F992CD31C8A2CD30137
:100910005315B62C531D8F2CD301D315B62CD31DD4
:10092000942CD3015316B62C531EB62CD301D314DA
:10093000B62C531D9E2CD3015316B62CD31DA32CBD
:10094000D3015316B62C531EB62CD301D314B62C98
:10095000D31CAD2CD3015315B62C531DB22CD3018F
:10096000D315B62C531EB62CD30153158F21400836
:10097000C4004108C5005F18DF145F1CDF10480881
:10098000C9000C304A05031D05120C304B05031D30
:1009900085120C304C05031D05100C304D05031D50
:1009A00085100C304E05031D87100C304F05031DBC
:1009B00007110C305005031D07100C305105031DA5
:1009C00087120C305205031D07120C305305031D0E
:1009D000871149080E020318192D12304A05031D0C
:1009E000051612304B05031D851612304C05031DEC
:1009F000051412304D05031D851412304E05031DDC
:100A0000871412304F05031D071512305005031DC2
:100A1000071412305105031D871612305205031DAD
:100A2000071612305305031D8715FF3048020319BE
:100A300008008F08031D08008E2049080E02031CC1
:100A4000192D18304A05031D051206304A05031DED
:100A5000051618304B05031D851206304B05031D86
:100A6000851618304C05031D051006304C05031D76
:100A7000051418304D05031D851006304D05031D66
:100A8000851418304E05031D871006304E05031DD2
:100A9000871418304F05031D071106304F05031D3D
:100AA000071518305005031D071006305005031DAB
:100AB000071418305105031D871206305105031D18
:100AC000871618305205031D071206305205031D04
:100AD000071618305305031D871106305305031DF3
:040AE000871508006E
:084000000400030002000600A9
:02400E00CC33B1
:10420000010003000300030003000200020002009B
:104210000200000000000000000003000300FF0097
:10422000020000000000000000000000000000008C
:104230000000C000C000C000C000C000C000FF00FF
:10424000FF00C300F300CF00FF00C300F300CF0066
:10425000FF00C300F300CF00FF00C300F300FF0026
:104260000100FF00FF00FF00FF00FF00FF00FF0054
:10427000FF00FF00FF00FF00FF00FF00FF00FF0046
:10428000FF00FF00FF00FF00FF00FF00FF00FF0036
:10429000FF00FF00FF00FF00FF00FF00FF00FF0026
:1042A000FF00FF00FF00FF00FF00FF00FF00FF0016
:1042B000FF00FF00FF00FF00FF00FF00FF00FF0006
:1042C000FF00FF00FF00FF00FF00FF00FF00FF00F6
:1042D000FF00FF00FF00FF00FF00FF00FF00FF00E6
:1042E000FF00FF00FF00FF00FF00FF00FF00FF00D6
:1042F000FF00FF00FF00FF00FF00FF00FF00AA001B
:00000001FF
